:020000040000FA
:100000003C280000000000003C2882070034003437
:100010000034003400340034003400340034003440
:100020000034003400340034003400340034E83448
:100030007134E4347234E2347434E1347834D834D2
:10004000B134D434B234D234B434D134B8340034CA
:10005000003400340F39820701340234033404348D
:10006000063408340B341034173420342D34403423
:100070005A348034B434FF3483168B0196013930FE
:100080008500870170309F009101111483120130A7
:100090009F00A701A901850187019F1495202414C1
:1000A0000830A500A6010310260E0E39A30026086D
:1000B0001F39A8001230A200230829070520A0003C
:1000C000A00CA10CA00CA10CA10CA10E8501200874
:1000D000870021088500A30AA20B5C28A70A1F300D
:1000E000A705A91028082702031CA9148501870168
:1000F00087099F1853288D2024188028A6008B2854
:10010000A50B8B280830A500A60A8D202602031C0B
:1001100053282410A6039F1453281E09A00003107F
:10012000200C20070318FF30080085018701F030FC
:10013000BA20A701FF30A5003830870087101030A3
:10014000A80028032A20A700871400008710A00118
:1001500003140630A000A00BAB28A70BA928A50B01
:10016000A128FF30A5000310A80BA1289F149F18F9
:10017000B7280800A2002C30C020A20BBC28080021
:0C018000AA00AB0BC128AA0BC128080084
:04018C000034003407
:02400E00D33CA1
:04420000DB000300DC
:00000001FF
